:020000000528D1
:06000A008316FF308600A2
:10001000FE308500D030810020308B00831200300C
:100020009000910092009300940095009600970034
:10003000980099009A009B00FF30061890008618DF
:1000400091000619920086199300061A9400861AE8
:100050009500061B9600861B9700851898000519C9
:10006000990085199A00051A9B00051405140510BE
:100070000000000000000000000000000000000080
:100080000000000000000000000000000000000070
:100090000000000000000000000000000000000060
:1000A0000514051405100000000000000000000009
:1000B0000000000000000514051405141030840031
:1000C000000805108500000000000000000000008E
:1000D0000000000005140514051403116400840ACF
:0A00E00004081C3A031D60280F28D5
:00000001FF
